:100000000C94C7020C94FF020C94FF020C94FF02A4
:100010000C94FF020C94FF020C94FF020C94FF025C
:100020000C94FF020C94FF020C94EC220C94BE235F
:100030000C94FE1D0C94FF020C94FF020C94FF0222
:100040000C94FF020C94FF020C94FF020C94FF022C
:100050000C94FF020C94861E0C94FF020C94FF0279
:100060000C94FF020C94FF020C94FF020C94FF020C
:100070000C94FF020C94FF020C94FF020C94FF02FC
:100080000C94FF020C94FF020C94FF020C94FF02EC
:100090000C94FF020C94FF020C94FF020C94FF02DC
:1000A0000C94FF020C94FF020C94FF02A505A50519
:1000B000D105D10539066407640764075706F006C1
:1000C000010701072B2452244A2552244A259E2445
:1000D000C1244A2518252725290000003A003B00A5
:1000E0003C003D003E003F00400041004200430014
:1000F0004400450046004700480035001E001F0030
:1001000020002100220023002400250026002700D3
:100110002D002E002A0049004A004B002B0014003D
:100120001A000800150017001C0018000C0012002F
:1001300013002F00300028004C004D004E00390005
:1001400004001600070009000A000B000D000E0055
:100150000F003300340032000000000000000000F7
:10016000E10064001D001B000600190005001100DD
:100170001000360037003800E50000000000520093
:100180000000E0000000E2000000000000000000AD
:100190002C0000000000E7000000015150000000AA
:1001A00051004F00010000000100010001000100AA
:1001B0000100010001000100010001000100010037
:1001C0000100010001000100010001000100010027
:1001D0000100010001000100010001000100010017
:1001E0000100010001000100010001000100010007
:1001F000005C01000100010001000100010001009C
:1002000001000100CE5CCF5C010001000100010093
:1002100001000100010001000100010001000100D6
:1002200001000100000000000000000001000100CA
:1002300001000100010001000100010001000100B6
:1002400001000100010000000000C65C0000010088
:10025000000001000000000000000000010000009C
:100260000000010000000100C95C0000C75CCA5C1E
:1002700000047F3F1F643214643214783C1E1E1445
:100280000A052223252628292A2C2D2F3032333502
:1002900036383A3B3D3E4042434547494A4C4E5032
:1002A00051535557595A5C5E6062646668696B6D5C
:1002B0006F71737577797B7D7F81838587898A8C60
:1002C0008E90929496989A9C9E9FA1A3A5A7A8AA67
:1002D000ACAEAFB1B3B4B6B8B9BBBCBEBFC1C2C39C
:1002E000C5C6C7C9CACBCCCDCED0D1D2D2D3D4D536
:1002F000D6D7D7D8D9D9DADADBDBDBDCDCDCDCDC5F
:10030000DDDDDDDDDCDCDCDCDCDBDBDBDADAD9D936
:10031000D8D7D7D6D5D4D3D2D2D1D0CECDCCCBCAC4
:10032000C9C7C6C5C3C2C1BFBEBCBBB9B8B6B4B3EA
:10033000B1AFAEACAAA8A7A5A3A19F9E9C9A989680
:100340009492908E8C8A89878583817F7D7B797753
:100350007573716F6D6B6968666462605E5C5A5933
:1003600057555351504E4C4A4947454342403E3DF4
:100370003B3A3836353332302F2D2C2A2928262582
:100380002322FFAA7F554000010101010101010163
:100390000102020202020202020203030303030338
:1003A0000303040404040404040505050505060606
:1003B00006060607070707070808080809090909C4
:1003C0000A0A0A0B0B0B0C0C0C0D0D0D0E0E0E0F6A
:1003D0000F0F1010111111121213131414151516FA
:1003E000161717181819191A1A1B1B1C1D1D1E1E6B
:1003F0001F202021222223242425262627282929BC
:100400002A2B2C2D2D2E2F303132323334353637E6
:1004100038393A3B3C3D3E3F4041424344454647E4
:1004200048494A4C4D4E4F50515354555658595ABD
:100430005B5D5E5F616264656668696B6C6D6F7061
:1004400072737577787A7B7D7E8082838587888AD0
:100450008C8E8F91939596989A9C9EA0A2A3A5A707
:10046000A9ABADAFB1B3B5B7BABCBEC0C2C4C6C903
:10047000CBCDCFD1D4D6D8DBDDDFE2E4E7E9EBEEBC
:10048000F0F3F5F8FAFDFF24034100630065002056
:10049000006F00660020005300700061006400657A
:1004A000007300200054004B004C0000001C03416E
:1004B000006300650020006F00660020005300709C
:1004C0000061006400650073000000040309040972
:1004D000023B00020100A0FA09040000010301012F
:1004E00000092111010001224000070581030800D5
:1004F00001090401000103000000092111010001AC
:1005000022320007058203200001120100020000D0
:1005100000084B5000100100010200010501098094
:10052000A101850319012AB700150126B70095011D
:1005300075108100C0050C0901A101850419012A6B
:10054000A002150126A002950175108100C00501C9
:100550000906A101050719E029E7150025019508FD
:10056000750181029501750881010507190029FFB0
:10057000150026FF00950675088100050819012958
:1005800005950575019102950175039101C011242E
:100590001FBECFEFDAE0DEBFCDBF04B603FE18C04A
:1005A0008091F4039091F503A091F603B091F703C5
:1005B0008730904BA740B04B59F41092F40310923F
:1005C000F5031092F6031092F703E0E0F8E30995C3
:1005D00011E0A0E0B1E0EAEFFCE402C005900D926A
:1005E000A23CB107D9F723E0A2ECB1E001C01D9213
:1005F000A43FB207E1F70E94A3130C947B260C944E
:10060000000081E0089581E008950C9403030895AB
:100610000C9407031F93CF93DF9300D000D01F9259
:10062000CDB7DEB749835A836B833091C501898189
:100630009A81311114C0662359F0222349F00E9497
:100640009D09182F682F89819A810E94460903C04D
:100650000E947109182F69817A81812F04C00E943C
:100660009D0969817A810F900F900F900F900F90E4
:10067000DF91CF911F910C94ED10FC01262F40814A
:1006800051816281738184810C940A0381E0089511
:10069000CF93DF93EC0160E00E943D03BE01DF9148
:1006A000CF910C9408030C9436120C9432120895D6
:1006B0000E94F0070E9457032FEF84E39CE0215033
:1006C00080409040E1F700C000000C94AC1E0F93F6
:1006D0001F93CF93DF938C0161E00E943D03EC01F7
:1006E000B8010E940503882309F444C0B801CE0173
:1006F0000E94D51C8823F1F1B801CE010E94E91AAD
:100700008823C1F1B801CE010E94311C882391F1E8
:10071000B801CE010E94EF19882361F1F8018281AE
:10072000882309F1CB358DE5D807C1F050F4C11508
:10073000FCE5DF0781F0CF3DDC45A9F40E94D40E33
:1007400019C0CC35EDE5DE0761F0CD35DD4559F456
:100750000E94170E08C00E9458030CC00E94200E71
:1007600002C00E94230EC801DF91CF911F910F910B
:100770000C94010380E0DF91CF911F910F910895B8
:100780000E94DE1D0C94D9030E94DC030C94E41D2E
:1007900008950C94C80381E008950C94CB03089548
:1007A000CF93C82F0E94C9038C2F0E94CD03CF91F5
:1007B000089580E00C94D0030E94311D0C94D00366
:1007C0000E94311D9091C401891721F08093C401CA
:1007D0000C94D0030895CF93DF93CDB7DEB72B975A
:1007E0000FB6F894DEBF0FBECDBF4F835887698721
:1007F0007A878B8761110E94630D9E012F5F3F4FA7
:1008000086E0F90111928A95E9F785E0FE013796B5
:10081000D90101900D928A95E1F789819A814C81E5
:100820005D81452B31F09F3F31F491E08F3F19F40A
:1008300003C091E001C090E090FF09C049815A8156
:100840006B817C818D819E810E94840C05C0C901D1
:100850000E9446038111F2CF2B960FB6F894DEBFAB
:100860000FBECDBFDF91CF910895FC0180819181B2
:100870000E94DF090895CF93882309F49CC0C82FF4
:100880008238C1F40E94311D81FD95C069E38091D9
:100890000201909103010E94B61D0E94850D2FEF69
:1008A00081EE94E0215080409040E1F700C00000CC
:1008B00069E319C0833801F50E94311D80FD7BC0BA
:1008C00063E580910201909103010E94B61D0E9490
:1008D000850D2FEF81EE94E0215080409040E1F7AC
:1008E00000C0000063E580910201909103010E9425
:1008F000B81DCF910C94850D8438C1F40E94311D30
:1009000082FD59C067E480910201909103010E9429
:10091000B61D0E94850D2FEF81EE94E0215080409E
:100920009040E1F700C0000067E4DDCF8CEF8C0F52
:10093000813AD0F46C2F80910201909103010E94C2
:10094000801D882349F06C2F809102019091030152
:100950000E94B81D0E94850D6C2F8091020190911C
:1009600003010E94B61DC5CF80E28C0F883048F489
:10097000C77081E001C0880FCA95EAF70E94460D52
:10098000B8CFEBE5EC0FE33040F4F0E0EE5AFE4F69
:10099000808190E0CF910C94481DC85AC73158F41B
:1009A000EC2FF0E0EE0FFF1FEC5DFE4F8081918198
:1009B000CF910C945E1DCF910895882309F45BC0FC
:1009C000682F823879F40E94311D81FF54C069E399
:1009D00080910201909103010E94B61D0E94850D35
:1009E00069E310C08338B1F40E94311D80FF43C019
:1009F00063E580910201909103010E94B61D0E945F
:100A0000850D63E580910201909103010E94B81D5C
:100A10000C94850D843879F40E94311D82FF2BC01F
:100A200067E480910201909103010E94B61D0E942B
:100A3000850D67E4E7CF8CEF860F813A18F380E2EB
:100A4000860F883048F4677081E001C0880F6A958E
:100A5000EAF70E944C0DDCCF8BE5860F833020F443
:100A600080E090E00C94481D685A673120F480E0E3
:100A700090E00C945E1D08951F93CF93DF93182F81
:100A8000EB010E943B04209741F08FE99FE0019722
:100A9000F1F700C000002197F6CF812FDF91CF91B1
:100AA0001F910C94DD04893319F060E070E002C0FE
:100AB00060E570E00C943C05882321F00E94460D0F
:100AC0000C94850D0895882321F00E944C0D0C9400
:100AD000850D0895CF92DF92EF92FF920F931F93AF
:100AE000CF93DF937C01D62FC72FFC0112810581A4
:100AF00002950F700E943C0D8823B9F01123A9F0D4
:100B00008C2F807F803421F080E28D0F883068F058
:100B10008091A50282FD09C082E00E94E50D0E943D
:100B20003C0D91E0D82ED92601C0D12CCC2EC294F8
:100B30008FE0C8228C2D90E08C30910508F0C4C164
:100B4000FC01EA5AFF4F0C94D6258C2F807FCF7082
:100B5000882311F0C295C07F112399F0CC2309F4AA
:100B60009FC180E28D0F883010F0D11104C08C2F0E
:100B70000E94460D03C08C2F0E94560D0E94850DC9
:100B80008FC18D2F0E94DD04CC2309F49DC180E22A
:100B90008D0F883038F1DD2329F18C2F0E945C0DF8
:100BA00024C08C2F807FCF70803211F0C295C07F1F
:100BB000DD2319F0D130A1F13DC08091A50282FF63
:100BC00017C0112349F0CC2329F08C2F0E94460D29
:100BD0000E94850D80E065C180E00E94DD04CC2389
:100BE00009F472C18C2F0E944C0D0E94850D6CC1BE
:100BF000112371F0002341F0013031F40E94660DA1
:100C00008C2B0E946E0D60C10E94660D8C2B1DC046
:100C1000002319F0013009F457C10E947B0D25C053
:100C2000112321F0063008F04FC10EC0053008F046
:100C30004BC11BC0112361F0002331F0F701858106
:100C400080FF2EC18F7085838C2F0E945C053CC174
:100C5000002359F0D93309F034C1FFEF07EE13E058
:100C6000F15000401040E1F72AC18C2F0E9463052B
:100C70002BC18C2F86958695837019F0813061F099
:100C800023C1112321F08D2F9C2F937002C080E08F
:100C900090E00E94481D20C1112321F08D2F9C2F30
:100CA000937002C080E090E00E945E1D15C18C2F01
:100CB000837009F047C011110BC12D2F2295269585
:100CC0002770220F220F6D2F6F70862F90E0A0E00B
:100CD000B0E0022E04C0880F991FAA1FBB1F0A9400
:100CE000D2F7D4FF10C04FE050E060E070E004C0E5
:100CF000440F551F661F771F2A95D2F740955095D0
:100D00006095709503C040E050E0BA01C695C69565
:100D1000C3708A019B01082B192B2A2B3B2BC9017D
:100D2000B801C23049F058F4C13019F00E945C0893
:100D3000CFC00E944A08CCC00E946E08C9C00E9461
:100D40004808C6C0112319F08C2F817001C0869508
:100D5000882309F4BDC02D2F229526952770220FD8
:100D6000220F6D2F6F70862F90E0A0E0B0E0022E72
:100D700004C0880F991FAA1FBB1F0A94D2F7D4FF83
:100D800010C04FE050E060E070E004C0440F551F19
:100D9000661F771F2A95D2F74095509560957095FC
:100DA00003C040E050E0BA01C695C695C3708A0101
:100DB0009B01082B192B2A2B3B2BC901B801C230F0
:100DC00049F058F4C13019F00E94210981C00E94F5
:100DD0000F097EC00E9433097BC00E94820878C040
:100DE000CF70112339F08C2F0E94A8088D2F0E94FC
:100DF0005C056EC08D2F0E9463058C2F0E94C90870
:100E000067C0D23F21F128F4D03F41F0D13FC1F07B
:100E100043C0D33F19F1D43F79F03EC0112341F0D4
:100E2000053008F051C08C2F8F710E94EE084CC025
:100E3000063008F049C0F7CF8091A50282FF18C0A4
:100E4000112339F08C2F8F710E94A8083DC0112307
:100E5000C9F38C2F8F710E94C90836C0112329F065
:100E60008C2F8F710E9493082FC00E948E082CC077
:100E7000112349F0CF718C2F0E94A80863E08C2FBA
:100E80000E94CA0D21C081E00E94E50D0230E0F011
:100E900082E00E94E50D18C0112331F0002391F289
:100EA0008D2F0E943B0410C0002399F2D93349F4DE
:100EB0001FEF27EE33E0115020403040E1F700C033
:100EC00000008D2F0E94DD0488EF8C0D843020F40B
:100ED0000E94311D0E94D003DD20C9F00E94380D10
:100EE00080FD15C0F70112820E94320D0E94A808F1
:100EF000C7010E94A8070E94320DDF91CF911F9178
:100F00000F91FF90EF90DF90CF900C94C908DF9184
:100F1000CF911F910F91FF90EF90DF90CF900895A8
:100F20000F931F93CF93DF93EC01688179818A81BE
:100F30000E94EA098C010E9445090E943608B80106
:100F4000CE010E946A05DF91CF911F910F91089504
:100F5000CF93DF93EC01988189812B813C81232BF6
:100F600031F08F3F31F481E09F3F19F403C081E0FD
:100F700001C080E080FD1DC0CE010E946703811189
:100F800010C00E943C0D8823A1F08A81882389F03B
:100F90008091A50282FD0DC082E0DF91CF910C947B
:100FA000E50DCE010E949007CE01DF91CF910C9408
:100FB0004803DF91CF91089580E090E00E94481DA2
:100FC00080E090E00E945E1D0E94630D0C94850DF0
:100FD00080910201909103010E94BA1D0C94DC07DC
:100FE0000E94530D0C94E80792959F70963079F00B
:100FF00010F4925001C09A50923068F4803F69F02A
:1010000018F4883E40F409C0843F29F406C0883EA5
:1010100020F0813F11F080E0089581E00895FC0107
:10102000808191810E94DF090E94F4070895CF9387
:10103000DF9300D000D01F92CDB7DEB70F900F9096
:101040000F900F900F90DF91CF910895CF93DF9382
:1010500000D000D000D0CDB7DEB726960FB6F894FA
:10106000DEBF0FBECDBFDF91CF91089508950895E3
:101070000C9437080C9438080E943A0860930B02CD
:1010800070930C0280930D0290930E020C94DC0777
:101090000C943C080F931F9300910B0210910C02CB
:1010A00020910D0230910E02602B712B822B932B1D
:1010B0001F910F910C943C080F931F9300910B020A
:1010C00010910C0220910D0230910E0260237123C9
:1010D000822393231F910F910C943C080F931F932D
:1010E00000910B0210910C0220910D0230910E0222
:1010F00060277127822793271F910F910C943C083A
:101100000C9437080E9480086093070270930802CD
:101110008093090290930A020C94DC0760E070E06F
:10112000CB010C9482080F931F9341E050E060E0E4
:1011300070E08A019B0104C0000F111F221F331FA2
:101140008A95D2F7C901B8011F910F910C948208BA
:101150000F931F9341E050E060E070E004C0440F43
:10116000551F661F771F8A95D2F7809107029091CD
:101170000802A0910902B0910A028A019B01082B82
:10118000192B2A2B3B2BC901B8011F910F910C94ED
:1011900082080F931F9341E050E060E070E004C0CC
:1011A000440F551F661F771F8A95D2F740955095BB
:1011B000609570958091070290910802A0910902B4
:1011C000B0910A028A019B01082319232A233B2399
:1011D000C901B8011F910F910C9482080F931F93BE
:1011E00041E050E060E070E004C0440F551F661F0E
:1011F000771F8A95D2F78091070290910802A091FB
:101200000902B0910A028A019B01082719272A279F
:101210003B27C901B8011F910F910C9482080F93CD
:101220001F9300910702109108022091090230914A
:101230000A02602B712B822B932B1F910F910C9420
:1012400082080F931F9300910702109108022091CA
:10125000090230910A0260237123822393231F9194
:101260000F910C9482080F931F9300910702109125
:1012700008022091090230910A0260277127822713
:1012800093271F910F910C948208089521E1929F5A
:10129000800D1124E82FE695E695E695877051E0DC
:1012A00001C0550F8A95EAF785E0E89FF001112407
:1012B000EA53FE4F20E030E070E04081CB01022E87
:1012C00002C0969587950A94E2F7817081958427EC
:1012D0008523842781932F5F3F4F2530310569F7A0
:1012E000089521E1929F800D1124682F66956695DF
:1012F0006695982F977085E0689FB001112440E0B3
:1013000050E080E0FB01E40FF51FEA53FE4F20811F
:1013100030E0092E02C0369527950A94E2F7217035
:101320003327042E01C0220F0A94EAF7822B4F5F65
:101330005F4F4530510531F70895BF92CF92DF924C
:10134000EF92FF920F931F93CF93DF938C01C09086
:101350000702D0900802E0900902F0900A02809102
:101360000B0290910C02A0910D02B0910E02C82ABE
:10137000D92AEA2AFB2ACFE1D0E0D701C6010C2EF8
:1013800004C0B695A795979587950A94D2F780FDE6
:1013900004C0219790F7B12C07C0BC2EB8018C2F48
:1013A0000E9400110197A9F38B2DDF91CF911F911E
:1013B0000F91FF90EF90DF90CF90BF900895CF9363
:1013C000DF93EC010E949D09BE010E940011DF9194
:1013D000CF9108951F93CF93DF93EB019091C501B7
:1013E000992321F0CB010E94DF0913C0882349F023
:1013F000CB010E949D09182F682FCE010E9446093B
:1014000004C0CB010E947109182FBE01812F0E94D8
:101410000011DF91CF911F9108951F93CF93DF9318
:10142000C0910F0216E080911002C81799F0D0E029
:101430001C9FF0011D9FF00D1124EF5EFD4F4081B8
:10144000518162817381848195810E942608219651
:10145000C770E9CFDF91CF911F910895409141026C
:101460005091420260914302709144028091450282
:10147000909146020C942608EF92FF920F931F93CF
:10148000CF93DF938091460282958F7009F065C0FB
:1014900080914302882309F460C080910F02F0908C
:1014A0001002109141020091420260914402709139
:1014B000450291E01F3F09F090E0C0910001D091FA
:1014C0000101292F96E0E92E8F1509F446C0611518
:1014D000710521F00F3F21F030E003C031E001C081
:1014E000322F90E030FD36C0E89EF001E99EF00D0D
:1014F0001124DF01AF5EBD4F11963C91119730135F
:1015000029C03C91311326C012963C91129731119B
:1015100021C013964D915C911497461B570B4C17A5
:101520005D07C0F4809146028F708061809346020F
:10153000EA5EFD4F80818F708061808381E492E05C
:101540000E94A807DF91CF911F910F91FF90EF901C
:101550000C940D0A01968770B7CFDF91CF911F9140
:101560000F91FF90EF9008959F92AF92BF92CF920C
:10157000DF92EF92FF920F931F93CF93DF93CDB73C
:10158000DEB761970FB6F894DEBF0FBECDBF8C01FA
:1015900085E0F801DE011D9601900D928A95E1F734
:1015A000D8011296EC9090914102E0914202209174
:1015B0004402309145022115310531F0EF3F31F4FD
:1015C00081E09F3F19F403C081E001C080E0B82FA3
:1015D000B1709B2E80FD47C1D8014C9111965C9152
:1015E00011971396AD90BC90149781E4C82E82E0B9
:1015F000D82EF0904302B501621B730B20910001BD
:1016000030910101FF2009F4D9C080914602621790
:10161000730708F095C0282F207F09F052C05E1391
:1016200013C0491311C0FE2CE1100EC08F708061F1
:10163000809346020E942E0AC6010E94A80780914C
:101640004602F80185834DC1AB2831F05F3F31F48C
:1016500081E04F3F19F403C081E001C080E080FDCC
:1016600003C081E08E2502C080E090E0F82FF17089
:10167000FF2E80FF1CC080910F022091100236E0E7
:10168000821709F40BC190E0389FF001399FF00DEB
:101690001124EF5EFD4F6181561306C06081461331
:1016A00003C06281E61203C001968770E9CFFE2C69
:1016B000EE2009F416C180914602816080934602B3
:1016C00054C05E1306C0491304C0E11002C0F80103
:1016D00099C0C8010E940F08882361F1EE2051F1E2
:1016E00020914602822F82958F7090E0029774F0CD
:1016F000809141029091420298878F831986BB8620
:10170000AA862C87CE0107960E94A80786E0F801DA
:10171000A1E4B2E001900D928A95E1F70E943C0AA3
:101720000E942E0A0AC05E1711F1C8010E940F081C
:1017300081112CC0C8010E94A807FF24F394D1C0D6
:10174000282F207F81F77A2DB98AA88A6E2D898962
:101750000E94170881E492E00E94A80786E0D60163
:101760001D928A95E9F70E942E0AF12CBAC04913FE
:10177000DCCFE110DACFF8018583C8010E94A80709
:1017800086E0D6011D928A95E9F7ABC0EE2091F272
:1017900020914602822F82958F7090E002970CF480
:1017A000B5CF80914102909142029A8389831B8236
:1017B000BD82AC822E83CE010196A6CF621773073D
:1017C00008F044C0FE2CEE2009F4B4CF5E1330C004
:1017D00049132EC02091460220FD21C0822F829500
:1017E0008F70482F50E041155105C9F0F80125834D
:1017F0004F30510541F08F5F982F9295907F822F47
:101800008F70892B8583C8010E94A80786E0F801A4
:10181000A1E4B2E001900D928A95E1F73CC086E028
:10182000F801A1E4B2E001900D928A95E1F759C068
:10183000C8010E940F08811169CF80914602816022
:1018400080934602C8010E94A8074BC07A2DB98A2E
:10185000A88A6E2D89890E94170886E0D6011D92FC
:101860008A95E9F718C0EE2009F464CFC8010E94F8
:101870000F08F82E882309F45DCF86E0F801A1E473
:10188000B2E001900D928A95E1F781E492E00E9426
:1018900035040E943C0A0E942E0A23C04D875E87B1
:1018A0008D859E850E94DF09292F22952F70223079
:1018B00028F49F7039F0811105C00BC0243028F442
:1018C0009F7049F4805E883020F0C8010E94A8070C
:1018D0009F2CF92C06C0D80115969C91907F91F70A
:1018E000F8CF8F2D61960FB6F894DEBF0FBECDBF37
:1018F000DF91CF911F910F91FF90EF90DF90CF90EC
:10190000BF90AF909F9008951F93CF93DF93CDB773
:10191000DEB72C970FB6F894DEBF0FBECDBF4F8356
:10192000588769877A878B879C87CE0107960E94A4
:10193000B40A8823D1F09F8188852A853B85232B93
:1019400031F08F3F31F481E09F3F19F403C081E013
:1019500001C080E080FD47C04F81588569857A8548
:101960008B859C850E9426083EC086E0FE01379646
:10197000DE01119601900D928A95E1F7FF81E885CD
:101980006A857B856115710531F0EF3F31F481E0A7
:10199000FF3F19F403C081E001C080E080FD23C057
:1019A0002091100230E0C90101968770992740917B
:1019B0000F0250E084179507F1F1F983EA837D83E4
:1019C0006C8396E0929FD001939FB00D1124AF5E7F
:1019D000BD4FFE01319601900D929A95E1F78093EB
:1019E00010020E940D0A16E080910F0290911002E1
:1019F000891771F1189FC00111248F5E9D4F0E94BD
:101A0000B40A882329F1E0910F021E9FF0011124EE
:101A1000EF5EFD4F408151816281738184819581A8
:101A20000E94260880910F0290E001968770992706
:101A300080930F02D9CF0E94F007109210021092EB
:101A40000F02E1E4F2E086E0DF011D928A95E9F7FA
:101A50002C960FB6F894DEBF0FBECDBFDF91CF91AD
:101A60001F91089580914F028595859585950895DC
:101A700080914F028770089590914F02977081E096
:101A800009F480E0089580915A02089590915A02D5
:101A9000892B80935A020895809590915A02892348
:101AA00080935A02089510925A0208959091590213
:101AB000892B80935902089580959091590289232A
:101AC000809359020895109259020895809150020E
:101AD000089508950C94690D0C946A0D9091A502D7
:101AE00092FD08C090915002981721F08093500207
:101AF0000C946C0D089580915002882329F0109267
:101B0000500280E00C946C0D0895CF93DF93E09128
:101B10000201F091030180915A028083E091020159
:101B2000F0910301908180915902892B80838091EB
:101B30005002882381F0E0910201F091030190812D
:101B4000892B808380910201909103010E94741D72
:101B500081110E947B0DC0910201D091030148E0E8
:101B600050E067E472E0CE010E942626892B69F0DE
:101B700088E0FE01A7E4B2E001900D928A95E1F7BA
:101B8000CE01DF91CF910C943D1DDF91CF9108954F
:101B90000C94690D9091A50292FD10C098E0899F68
:101BA00090011124262B20934F020E94A8088091B7
:101BB0004F028595859585950C94C80D0C94A808C1
:101BC00010924F0280E00C94C80D20914F02809536
:101BD000822380934F02982F977099F430E0482F1A
:101BE000082E000C550B2417350759F09091A502CB
:101BF00092FD07C08595859585950E94C9080C942E
:101C0000E00D08959091A50292FB222720F9281754
:101C100069F080FB92F99093A5028091A4029091C3
:101C2000A5020E94500E82E00C94E50D089580916B
:101C3000A50282FB882780F991E089270C94020E87
:101C400081E00C94020E80E00C94020E6FEF7FEFA7
:101C500080E090E00C94652680E090E00E944126B0
:101C600021E0893E9E4F09F020E0822F089582E016
:101C700090E00C94332683E090E00C943326CF93CD
:101C800084E090E00E943326C82F82E290E00E9418
:101C900033262C2F30E0A901582BCA01CF9108958B
:101CA000CF93C92F682F84E090E00E9447266C2FC5
:101CB00082E290E0CF910C944726AB01BC018FE00B
:101CC00090E00C945926AB01BC0183E190E00C94A8
:101CD000592660E070E0CB010C94630E60E070E088
:101CE000CB010E945D0E0C94690E69EE7EEF80E0E0
:101CF00090E00E94652660E082E090E00E94472626
:101D000060E083E090E00E94472610920B02109260
:101D10000C0210920D0210920E0260E084E090E03E
:101D20000E94472660E082E290E00E94472660E041
:101D300085E090E00E94472660E086E090E00E9407
:101D400047266FEF87E090E00E94472640E050E092
:101D5000BA0188E090E00E94592660E08DE090E0B2
:101D60000E94472640E050E0BA0188E190E00E94DE
:101D7000592660E087E190E00E94472640E050E06D
:101D8000BA018CE190E00E94592660E070E080E2A8
:101D900090E00E94652640E050E0BA0188E190E0C2
:101DA0000E9459260C946E0E0C94750E682F8EE0CE
:101DB00090E00C9447260E946B1E6093770270930C
:101DC00078028093790290937A0260937302709301
:101DD00074028093750290937602089585B78068A7
:101DE00085BF85B7806885BF089581E008950C940C
:101DF000F50E08950C94F90E0C94F90E0C94FC0E4B
:101E00000C94F90E0C94000F0C94F90E0E94EE0E37
:101E10008CED91E10E94271D0E94040F0C94020F8B
:101E20000E94FA0E0C94F90E0E94F6110C94CF0346
:101E30000E94561E0E94FA120E94140F0E940E1950
:101E40000C94FE0E2F923F924F925F926F927F9270
:101E50008F929F92AF92BF92CF92DF92EF92FF92BA
:101E60000F931F93CF93DF93CDB7DEB72D970FB6A8
:101E7000F894DEBF0FBECDBF0E940F13282E811134
:101E80000E94DB0E8BE592E09D878C8700E010E0DE
:101E9000302E802F0E941A122B013C01EC85FD850B
:101EA00081919191A191B191FD87EC8753014201FC
:101EB00088269926AA26BB2681149104A104B10480
:101EC000B1F40F5F1F4F0630110511F78FEF8983B3
:101ED0008A831B820E945F1E8160782F9D838C8382
:101EE00049815A816B818D810E94EB0351C08091A1
:101EF0007B0281FD0E9426121B86C12CD12C76010B
:101F0000C394D501C4018C219D21AE21BF21892B11
:101F10008A2B8B2B91F10E94F70E8823D1F0FB8541
:101F2000FE833F824C205D206E207F2081E045288B
:101F30004628472809F480E088870E945F1E816058
:101F4000782F9A8789874E815F8168858A850E946C
:101F5000EB03000F111F000F111FF801E55AFD4F91
:101F600080819181A281B381C826D926EA26FB26E9
:101F7000C082D182E282F3820BC08B858F5F8B8718
:101F8000CC0CDD1CEE1CFF1C813109F0BACF99CFBF
:101F900081E0211001C080E02D960FB6F894DEBFDD
:101FA0000FBECDBFDF91CF911F910F91FF90EF90AA
:101FB000DF90CF90BF90AF909F908F907F906F9069
:101FC0005F904F903F902F9008950E94220F0E94A3
:101FD00041190C94E003CF93DF930E940511EC01AB
:101FE000811522E59207E8F5811531E5930708F0A0
:101FF000B6C0883E910528F5803E910508F0E9C0FD
:10200000883A910570F4853A910508F07AC08130DC
:10201000910509F473C008F4D9C0049708F0D9C039
:10202000D5C08F3B910508F0D1C0C85AD0E0CC0F85
:10203000DD1FCB5ADE4F0990D881C02DCE019464AC
:10204000C9C0811540E5940708F069C0811550E4C6
:10205000950708F060C09A9581159F4108F4B9C0B2
:10206000B5C0811536E5930728F5811545E5940738
:1020700008F092C0811554E5950708F087C0AC01BF
:1020800043705527282F26952695C115D34508F06E
:102090006CC081E090E002C0880F991F4A95E2F77A
:1020A00040E2249F90011124EC01C22BD32BCE01DE
:1020B0009C6890C081152AE5920780F4811539E566
:1020C000930708F072C0811548E5940708F47EC0B4
:1020D000D82FCC27CE01806F906A7CC09056811596
:1020E000904208F073C08D2F8F710E949911DD27E7
:1020F000D0628F71AE01582BCA016CC081E090E0B4
:1021000069C0C55AD0E0CD57DE4F8881C82FD0E0D6
:10211000CE0190645FC0DF70CE01906A5BC074E056
:10212000969587957A95E1F7282F23703C2F337089
:1021300081E090E002C0880F991F3A95E2F79C6811
:10214000AC01522B9A019C2F9F709695969550E268
:10215000959FE0011124C9018C2B9D2B3BC0D82FEA
:10216000CC27CE01816F906A35C081E090E002C03B
:10217000880F991F4A95E2F750E2259F900111249C
:10218000EC01C22BD32BCE019A6824C0D82FCC27C8
:10219000CE01846F906A1EC00E9499118F7190E0E9
:1021A000D82FCC27CE01906215C08F700E94991154
:1021B00094E0D695C7959A95E1F7CF70D0E0DC2FE3
:1021C000CC27D0699E01282BC90104C080E090E093
:1021D00001C0CE01DF91CF91089526E6829FC00114
:1021E0001124FC0121E1729FE00DF11D1124E60F85
:1021F000F11DEE0FFF1FE852FF4F85919491089556
:102200000E94ED100E94EB0F08958238910569F14C
:10221000B0F48133910509F46DC048F48932910519
:1022200009F463C08A32910509F469C008958533C1
:10223000910509F455C089339105B9F00895833E9D
:10224000910569F138F4803E9105B1F0823E910527
:1022500009F10895863E9105A9F1873E9105B9F1EE
:10226000843E910509F064C023C02091A40220FDA2
:102270004FC021FD4DC008958091A40280FD44C04F
:102280008091A50280FF44C08091A40284FD42C0D9
:1022900083EE4DC08091A40282FF38C0F5CF8091BB
:1022A000A40282FD33C08091A50280FD31C0ECCF35
:1022B0008091A50281FF32C08091A40284FD2AC0D2
:1022C00087EE35C08091A40283FF26C0F5CF8091B0
:1022D000A40283FD21C08091A50281FD1FC0ECCF27
:1022E0008091A40285FD1CC01DC08091A40285FDC3
:1022F00019C016C08091A40286FD16C017C0809137
:10230000A40286FD13C010C089E311C082EE0FC085
:1023100080EE0DC080E00BC086EE09C084EE07C0E1
:1023200089E205C085E303C08AE201C081E390E051
:1023300008959091A40292FF0DC0282F2871283093
:1023400019F4877F846006C0282F2471243011F48B
:102350008B7F886093FF0DC0282F2871283119F4D6
:10236000877E846106C0282F2471243111F48B7E6E
:1023700088612091A50220FF0DC0382F38713830B8
:1023800019F4877F816006C0382F3171313011F424
:102390008E7F886021FF0DC0282F2871283119F405
:1023A000877E816106C0282F2171213111F48E7E34
:1023B000886194FD877E089580E008950C94260E30
:1023C0000E940F138FE39CE90197F1F700C0000012
:1023D0000E940F1380E00E941A1260FF04C00E9446
:1023E000DE110C94AC1E08950C94E0110E942C0E8A
:1023F000811102C00E94D40E0E94370E80937B028E
:102400000E943F0E9093A5028093A4020E94F411B3
:102410000E943B0E682F70E080E090E00E94480828
:1024200060910702709108028091090290910A025E
:102430000C94800824E0829FC0011124FC01E25426
:10244000FD4F60817181828193810895089580EAB2
:102450008A95F1F7089500C008950C942712089505
:102460000C942F120C9430120C942F120C943412E2
:10247000F894E82FE295EF70F0E031A1282F2F704B
:1024800081E090E001C0880F2A95EAF7982F909597
:10249000932391A392A1892B82A3789408950F93FB
:1024A0001F93CF93DF93C7E9D1E089918F3F11F05C
:1024B0000E94381281E0CD39D807B9F7C6E8D1E0DB
:1024C00007E911E089918F3F11F00E9438120C1733
:1024D0001D07C1F7DF91CF911F910F9108954F9282
:1024E0005F926F927F928F929F92AF92BF92DF9294
:1024F000EF92FF920F931F93CF93DF938C01C62F20
:10250000D0E0CE0189569E4F7C01FC0190819F3F17
:1025100009F460C0D62EF894E92FE295EF70F0E050
:1025200081A19F7021E030E001C0220F9A95EAF767
:10253000822B81A382A12095282322A378940E9434
:102540002B12E6E8F1E027E931E0412C512C320171
:102550004394812C912C540181918F3F99F0A82FA5
:10256000A295AF70B0E090964C9150E08F70BA0198
:1025700002C0759567958A95E2F760FD03C0D301A7
:10258000C20103C080E090E0DC01882A992AAA2ACF
:10259000BB2A440C551C661C771C2E173F07E1F61E
:1025A000F70180818F3F11F00E94381261E08114A1
:1025B0009104A104B10409F460E08D2D0E942D1254
:1025C000CC0FDD1FCC0FDD1FC00FD11F8882998279
:1025D000AA82BB82DF91CF911F910F91FF90EF9064
:1025E000DF90BF90AF909F908F907F906F905F90A3
:1025F0004F9008950E944F1288E1EEEBF2E0DF0168
:10260000982F1D929A95E9F7E6EAF2E0DF011D9214
:102610008A95E9F786E00E945A130C945303FF92BF
:102620000F931F93CF93DF93CDB7DEB768970FB6A5
:10263000F894DEBF0FBECDBF8E010F5F1F4F88E144
:10264000F80111928A95E9F7F12C6F2DC8010E94CB
:102650006F12F394F6E0FF12F8CF48E150E0B801B2
:1026600086EA92E00E942626FF24F394009709F45C
:10267000F12C892B41F088E1F801A6EAB2E0019043
:102680000D928A95E1F72F2D46E06EEB72E086EA17
:1026900092E00E945B130E9455038F2D68960FB63F
:1026A000F894DEBF0FBECDBFDF91CF911F910F9188
:1026B000FF9008950895FF920F931F93CF93DF9398
:1026C000F82ED92F8B01C42F222349F081E080936B
:1026D0007E020E945F1E90937D0280937C02809117
:1026E0007E028823F1F080917C0290917D020E940D
:1026F000771E0597B0F0EF2DFD2FD80180E090E018
:102700004C2F50E08417950754F4019111912191B9
:1027100031910D931D932D933D930196F3CF10921C
:102720007E02DF91CF911F910F91FF9008950E943B
:1027300044200E94180F0C9450200E9454200E94A4
:10274000E50F0C946E200E94FD1D0E942B200E941C
:10275000060F0E9497130E949D130E94100FFBCF3B
:10276000EF92FF920F931F93CF93DF938B01682F0C
:1027700011110AC0442329F0E82FF0E0E957FC4F7B
:102780006491762F862F75C0212F30E0E82FF0E07E
:10279000442321F0E957FC4FE491F0E046E0049F28
:1027A000C0011124CFEFD0E0BE010E948C254BEA7E
:1027B0004603C001479F900D1124800F911D800F8B
:1027C000911D982F990F890FAE01421B530B4E9FFD
:1027D000D0014F9FB00D5E9FB00D11249B2F189F0D
:1027E000A0011124452F55278E01041B150B0E9FA8
:1027F000A0010F9F500D1E9F500D11247E01E81A5D
:10280000F108E29E8001E39E100DF29E100D11244E
:10281000212F3327C21BD30BCE9F9001CF9F300DAA
:10282000DE9F300D112462307105A9F048F4611566
:10283000710569F061307105C9F48B2F752F0DC0DA
:102840006430710581F058F06630710579F47E2F9F
:102850008B2F932F0DC0832F7B2F9E2F09C08E2F80
:102860007B2F952F05C08E2F732F02C07E2F852FB3
:10287000692FDF91CF911F910F91FF90EF900895F5
:1028800041E00E94B013089508950E9440140895F5
:10289000CF93DF93762FE901682F842F0E94451490
:1028A000798368838A83DF91CF910895433308F059
:1028B00042E30C9448148091D602282F269530E0EC
:1028C0002115310519F48170826005C0253231056A
:1028D00024F0817088648093D6028091D90283337A
:1028E00018F082E38093D902089588E090E00C9478
:1028F0003B26CF92DF92EF92FF926B017C010E9408
:102900005B14B701A60188E090E0FF90EF90DF90A4
:10291000CF900C945926E6EDF2E083E0808311829B
:102920008FEF828382E3838314826081718182814D
:1029300093810C9479148091D60280FF02C0869511
:10294000089580E008959091DA02933018F49F5F23
:102950009093DA02882351F06091D6027091D702E9
:102960008091D8029091D9020C947914089581E055
:102970000C94A3149091DA02992319F0915090933A
:10298000DA02882351F06091D6027091D7028091CB
:10299000D8029091D9020C947914089581E00C9496
:1029A000BA1470E00C94BE1A609108018091D602AE
:1029B00080FF0AC08091070123E0829FC00111249B
:1029C00085529D4F0C94D1148091090190910A0178
:1029D000891780F7E82FF0E09F01220F331FE20FE5
:1029E000F31FE552FD4F1182108212828F5FF0CFEC
:1029F0009091D60290FF16C09091090120910A0192
:102A0000921770F4E92FF0E0DF01AA0FBB1FEA0F65
:102A1000FB1FE552FD4F8183608342839F5FF0CFB0
:102A20000C94D4140895CF93DF9300D01F92CDB7A8
:102A3000DEB79091D60290FF0AC09E012F5F3F4FF4
:102A40000E9456144B8169818A810E94F8140F906C
:102A50000F900F90DF91CF910895CF93DF93EC010A
:102A6000EC81F0E0EE57FD4F4491E6EDF2E062813B
:102A700081810E9413158C818F5F8C83DF91CF91B0
:102A80000895CF93DF93EC01E6EDF2E0438162819C
:102A90008C810E9413158C818F5F8C83DF91CF9185
:102AA00008950F931F93CF93DF9300D01F92CDB75C
:102AB000DEB78C0180917F0281110AC09E012F5FD9
:102AC0003F4F42E36FEF0E9456148A8180937F024A
:102AD000F8018481813051F028F0823061F4409116
:102AE0007F020AC080917F0240E007C060917F02B0
:102AF00040E080E003C040E080E060E00E94F81425
:102B0000F801848190E0019663E070E00E94A025C6
:102B100084830F900F900F90DF91CF911F910F91B1
:102B20000895AF92BF92CF92DF92EF92FF920F93F0
:102B30001F93CF93DF9300D01F92CDB7DEB7182F2E
:102B4000F62E042FE22E9091D60290FF6DC0E92F51
:102B5000E695AE2FB0E0A356BE4F8C9180938902CC
:102B60009E7F923061F49E012F5F3F4F812F0E9424
:102B700056144B8169818A810E94F81443C08230C7
:102B800019F40091D9023EC0863019F41091D70291
:102B900039C08930D9F38931A9F5E9518E2F817077
:102BA000D82EE695F0E0EE57FC4FA590B490C12CDE
:102BB000BB2460910B01C61618F52C2D30E0A29EA7
:102BC000C001A39E900DB29E900D112470E00E9452
:102BD0008C25812FD11002C0860F01C0861B9091D9
:102BE0000901290F311DA901440F551F240F351F5D
:102BF00025523D4F402F6F2D0E945614C394D9CFBC
:102C00000E94D4141093D702F092D8020093D902F4
:102C1000EE2051F06091D6027091D7028091D802D7
:102C20009091D9020E9479140F900F900F90DF912C
:102C3000CF911F910F91FF90EF90DF90CF90BF90B9
:102C4000AF900895E6EDF2E09181282F43816281F3
:102C500088E0890F0C94911581E00C942216E6ED22
:102C6000F2E09181282F4381628188EF890F0C94D3
:102C7000911581E00C942F16E6EDF2E0628128E0D8
:102C8000620F08F46FEF282F438181810C94911516
:102C900081E00C943C16E6EDF2E0628128E0621BD4
:102CA00008F460E0282F438181810C94911581E024
:102CB0000C944B16E6EDF2E0438128E0420F08F455
:102CC0004FEF282F628181810C94911581E00C9443
:102CD0005A16E6EDF2E0438128E0421B08F440E09A
:102CE000282F628181810C94911581E00C946916E2
:102CF00020E00C949115FF920F931F93CF93DF93D5
:102D0000EC01F12C0FEF10E060910B01F616F0F4DE
:102D1000809109012F2D30E0280F311DC901880F46
:102D2000991F280F391F25523D4F70E0C8010E949E
:102D3000A025962F8C814091D9026091D802F99EEE
:102D4000800D11240E945614F394DECF0E94D414F7
:102D50009A818C8190FF02C08F5F01C081508C836B
:102D6000DF91CF911F910F91FF900895AF92BF9285
:102D7000CF92DF92EF92FF920F931F93CF93DF9347
:102D8000FC01828180FF02C00FEF01C001E010E072
:102D900048E5A42E80910B01181708F043C08091DC
:102DA0000901C12ED12CE601C80FD11DCE01880F1B
:102DB000991FC80FD91FC552DD4F198218821A8278
:102DC00034E0E32EF12CB12C809181028B0D8935FA
:102DD0002CF06A2D0E947E25892F05C087FF03C035
:102DE00090910B01890F082E000C990BC816D9067B
:102DF00091F48091D9028E9DA0018F9D500D1124D8
:102E000055954795559547959E016091D8028091BB
:102E1000D7020E945614B00EF1E0EF1AF108A1F6A5
:102E20001F5FB8CF0E94D41480918102013031F429
:102E3000811102C080910B01815007C090E0019682
:102E400060910B0170E00E94A02580938102DF91C8
:102E5000CF911F910F91FF90EF90DF90CF90BF9097
:102E6000AF900895CF938091090190910A0189173D
:102E700070F4E82FF0E09F01220F331FE20FF31FE1
:102E8000E552FD4F1182108212828F5FF0CFC0E0B9
:102E900060910B01C617C0F5EC2FF0E070E0CF0198
:102EA0000E94A02520910901820F20918002022E0C
:102EB000000C330B90E0E217F307CCF020910601F1
:102EC000022E000C330B2E173F078CF09C01220FB3
:102ED000331F820F931F9C0125523D4F4091D90211
:102EE0006091D8028091D7020E9456140BC0FC0159
:102EF000EE0FFF1F8E0F9F1FFC01E552FD4F118249
:102F000010821282CF5FC4CF0E94D4142091050199
:102F100080918002820F8093800290910601920F2F
:102F20009093060119165CF4082E000C990B409141
:102F30000B0150E041505109841795071CF0219571
:102F400020930501CF9108958F929F92AF92BF92E7
:102F5000CF92DF92EF92FF920F931F93CF93DF9365
:102F60008C01FC014481C42FD0E09E01DE010E944F
:102F7000E4259B01AC010E94FA256B017C01E0E293
:102F8000F0E0EC1BFD0BA5E5B0E09B01AC010E945D
:102F9000FA254B015C019F01DF010E94DC259B01AA
:102FA000AC010E9405269B01AC012C0D3D1D4E1D60
:102FB0005F1DC501B4010E94B425C22FD22F2A3251
:102FC00028F4F3E02F9F900111240DC025E530E097
:102FD0002C1B3109C901880F991F280F391F37FF92
:102FE00002C02F5F3F4F35952795C22FC095F12C1A
:102FF00085E5E82EED1A80910B01F816C8F4F1FC76
:1030000002C08E2D01C08D2F909109012F2D30E02F
:10301000290F311DA901440F551F240F351F2552BB
:103020003D4F4C2F6091D8020E945614F394E3CF89
:103030000E94D414F8018481811102C091E003C080
:10304000803219F49FEF9093040190910401890F4D
:10305000F8018483DF91CF911F910F91FF90EF9042
:10306000DF90CF90BF90AF909F908F9008950F9377
:103070001F93CF93DF93EC0100E010E080910B01F0
:10308000282F30E00217130724F5909109019801C9
:10309000290F311DA901440F551F240F351F25523B
:1030A0003D4F869590E04C81081719071CF4442386
:1030B00031F002C0411103C04091D90201C040E08B
:1030C0006091D8028091D7020E9456140F5F1F4F63
:1030D000D5CF0E94D4148C8190E0019681709927FD
:1030E0008C83DF91CF911F910F910895E6EDF2E06F
:1030F00080818E7F808360817181828193810E9433
:10310000791410928A022FEF80E792E021508040DC
:103110009040E1F700C000000C94D4146091D602F6
:10312000669570E04BE050E08CE091E00E9419263B
:10313000892B19F481E080938A020E945F1E90938C
:1031400083028093820208959091D60290FF35C049
:103150009170811102C0926006C0853210F09864AF
:1031600002C0880F982B9093D602662351F060918D
:10317000D6027091D7028091D8029091D9020E9414
:1031800079146091D602669570E04BE050E08CE0D7
:1031900091E00E941926892B19F010928A0202C030
:1031A0000E948E1881E0809385024091D90260913F
:1031B000D8028091D7020C9478160895682F9091C8
:1031C000D602969581E0890F853208F081E00C9453
:1031D000A41881E00C94DE18682F9091D602969581
:1031E0008FEF890F09F484E20C94A41881E00C9409
:1031F000EC1861E00C94A418E6EDF2E080818160A7
:10320000808386950C94F9188091D60280FD0C94E9
:1032100076180C94FC1860E00C94A4188091880235
:1032200081112EC00E942C0E811104C00E94D40E68
:103230000E948B140E9475146093D6027093D7027B
:103240008093D8029093D9026E7F61F40E948B1410
:103250000E9475146093D6027093D7028093D802AF
:103260009093D9020E945B1410928A028091D60238
:1032700080FF03C086950E940B1981E0809388022D
:1032800008950F931F93CF93DF9380918A02882331
:1032900009F485C080918902E091D602E695E81B89
:1032A000E0938402823049F4F0E0E258FD4FE4916B
:1032B000CE2FD0E00DE215E149C0863049F4F0E0B0
:1032C000E558FD4FE491CE2FD0E001E415E13EC07A
:1032D000893051F4E695F0E0E858FD4FE491CE2FA7
:1032E000D0E00BE716E132C08F3051F4E695F0E004
:1032F000EB58FD4FE491CE2FD0E006EB16E126C04F
:10330000853149F4F0E0EE58FD4FE491CE2FD0E046
:1033100002E317E11BC0883181F0833239F4E0E722
:10332000F2E0C591D49101E515E110C0843251F469
:10333000C4EFD1E007E318E109C0C8E2D0E004EA35
:1033400017E104C0C0EDD7E004E414E180918502E8
:10335000882361F0109285020E945F1E9093830281
:103360008093820210928702109286020E945F1E52
:10337000E0918202F09183028E1B9F0B8F3F9F474B
:1033800070F4EC0FFD1FF0938302E093820282E859
:1033900092E0F801DF91CF911F910F910994DF9195
:1033A000CF911F910F910895882311F0FA0101C068
:1033B000FB010994CF93DF93C82FD62F0E949B1453
:1033C0008C1740F00E949B148D1720F4DF91CF9151
:1033D0000C94E9188C2FDF91CF910C94F9181F935E
:1033E000CF93DF93FB0112811111C3C0EC010E9446
:1033F000430D8272CD3CFCE5DF0709F49AC0A8F5C5
:10340000C73CECE5DE0709F476C0A8F4C43C9CE5B3
:10341000D90709F45FC028F4C33CDC4509F457C060
:1034200054C0C53C9CE5D90709F459C0C63CDC45ED
:1034300009F45CC04AC0CA3CFCE5DF0709F46AC075
:1034400050F4C83CECE5DE0709F45AC0C93CDC4541
:1034500009F45BC03AC0CB3C9CE5D90709F45FC0D6
:10346000CC3CDC4509F460C030C0C23DFCE5DF0760
:1034700009F46FC088F4CF3C9CE5D90709F460C01B
:1034800008F45CC0C03DFCE5DF0709F45CC0C13D49
:10349000DC4509F45BC019C0C53D9CE5D90709F4BA
:1034A00060C050F4C33DFCE5DF0709F455C0C43DDE
:1034B000DC4509F454C009C0C63D9CE5D90709F4B0
:1034C00055C0CE35DD4509F454C011E052C00E940C
:1034D00004194FC046EF58E169EE78E104C049EEA7
:1034E00058E166EF78E10E94D41943C049E356E100
:1034F0006CE276E1F8CF4CE256E169E376E1F3CF96
:1035000047E556E168E476E1EECF48E456E167E549
:1035100076E1E9CF45E756E166E676E1E4CF46E6B7
:1035200056E165E776E1DFCF4EEC54E167EB74E1FD
:10353000DACF47EB54E16EEC74E1D5CF81E017C0F0
:1035400065E082E010C068E086E00DC06EE089E0D2
:103550000AC064E18FE007C067E185E104C088E14B
:1035600006C062E289E10E94DA1903C083E20E9488
:10357000F918812FDF91CF911F9108956E9A2EB186
:103580002F7B3EB130644FB7F894FC01CB01880F1C
:10359000991F680F791F6E0F7F1FE617F70789F0D5
:1035A000819198E03EB9000000C087FF2EB9880FD6
:1035B000000000C000C000C02EB900C09A9591F76D
:1035C000ECCF4FBF8FE594E00197F1F700C000000A
:1035D0000895CF93DF93EC01FB018281882309F4E6
:1035E0003CC1C430FDE5DF0760F4CB3F9CE5D90763
:1035F00088F49E0122503C452431310508F02EC14B
:1036000009C0C236EDE5DE0729F0C63AFDE5DF0761
:1036100009F024C10E943F0E9093A5028093A4025A
:10362000C1318CE5D80709F4C6C008F042C0C930E2
:10363000ECE5DE0709F49BC000F5C5308CE5D80742
:1036400009F485C078F4C330ECE5DE0709F478C0EE
:1036500008F07AC0C230DC4509F0F5C08091A402C0
:103660008160EFC0C7309CE5D90709F478C008F045
:103670007AC08091A4028061E4C0CD30FCE5DF0710
:1036800009F487C058F4CB309CE5D90709F479C018
:1036900008F07BC08091A40288606FC0CF30FCE549
:1036A000DF0709F480C008F082C08091A402877F00
:1036B000C8C0CE3F9CE5D90709F471C000F5C531FB
:1036C000FCE5DF0709F485C068F4C3319CE5D90740
:1036D00009F475C008F095C00E94F0078091A4021B
:1036E0008F77AFC0CC3FFCE5DF07A9F108F054C0ED
:1036F000CB3FDC4509F0A7C08091A50240C0C23095
:10370000EDE5DE0709F489C058F4C1158DE5D80749
:1037100009F45AC008F069C08091A50282602FC0E8
:10372000C236EDE5DE0709F47CC0C63AFDE5DF07E9
:1037300009F481C0C330DD4509F085C080E06EC06A
:103740008091A40282607DC08091A40216C0809105
:10375000A402886076C08091A50282604FC08091EB
:10376000A40280626EC08091A40280646AC00E943C
:10377000F0078091A402806864C0846062C08160A8
:103780003DC08091A4028E7F5CC08091A4028D7F99
:1037900058C08091A40216C08091A50218C08091E3
:1037A000A5028D7F2BC08091A4028F7E4AC080919C
:1037B000A4028F7D46C08091A4028F7B42C080917D
:1037C000A402877F8B7F3DC08091A5028D7F8E7F75
:1037D00015C08091A40282FB222720F991E0922754
:1037E00090FB82F990FB83F92CC08091A502982F61
:1037F000909591708E7F892B90FB81F98093A50223
:1038000022C00E94F0078091A40287FB222720F9A2
:1038100091E0922790FB87F914C081E00E94D60EB8
:1038200012C08091A40284FB222720F991E0922704
:1038300090FB84F906C08091A402982F909590FB8C
:1038400080F98093A4028091A4029091A5020E9425
:10385000500E0E94F00780E001C081E0DF91CF911F
:103860000895CF93DF9386319C4541F5EB010E948B
:10387000430D982F8A812091020130910301882302
:1038800079F09A7A81E009F480E080938B029111BB
:1038900002C069E201C065E3C9010E94B61D0AC009
:1038A00080918B02811102C069E201C065E3C90108
:1038B0000E94B81D0E94850D80E001C081E0DF916B
:1038C000CF9108950F931F93CF93DF93C42FD22FDF
:1038D000FC0182818823C9F040938E020E945F1E02
:1038E00090938D0280938C0280E28C0F883008F0D8
:1038F00057C0C77081E001C0880FCA95EAF7DF9111
:10390000CF911F910F910C945C0580918E0248130A
:1039100030C080918C0290918D020E94771E883C6D
:10392000910538F510E21D0FCD17B9F080E28C0F2C
:10393000883040F4C77081E001C0880FCA95EAF76B
:103940000E946305183028F581E09D2F977001C013
:10395000880F9A95EAF70E945C05802F0E94530514
:103960001830F0F4D77081E001C0880FDA95EAF7DB
:103970000AC080E28C0F883098F4C77081E001C0E3
:10398000880FCA95EAF7DF91CF911F910F910C94A0
:103990006305802FDF91CF911F910F910C945305F8
:1039A000DF91CF911F910F9108950F939C01CB014F
:1039B000243F4CE5340731F188F4293DFCE53F070D
:1039C000D9F02A3D4CE5340779F1283D3C45A9F56D
:1039D00006E221EE41EE68ED7CE52BC0263FFCE5DA
:1039E0003F07E1F0A8F0273F3C4539F507E225EE17
:1039F00046EE67EF7CE51DC007E225EE45EE69ED7A
:103A00007CE517C006E221EE40EE64EF7CE511C0D4
:103A100007E225EE44EE65EF7CE50BC006E221EE01
:103A200042EE66EF7CE505C008E221E045EE6AED76
:103A30007CE50E94621C80E008C0FC018281882332
:103A400019F010928E0201C081E00F9108959093B9
:103A5000C3018093C20108959093940280939302CE
:103A60000895E0919302F0919402309721F0019033
:103A7000F081E02D099480E00895E0919302F091A7
:103A80009402309721F00280F381E02D099408958B
:103A900020919102309192022817390771F090938A
:103AA000920280939102E0919302F09194023097F8
:103AB00021F00680F781E02D0994089520918F026E
:103AC000309190022817390771F0909390028093FB
:103AD0008F02E0919302F0919402309721F00084DC
:103AE000F185E02D09940895FC01329697E080E07D
:103AF000915029F021912223D9F38F5FF9CF0895B6
:103B0000662349F0FC01329608962191621729F04C
:103B1000E817F907D1F780E0089581E008959C0146
:103B2000FC0132969FEF80E04191461789F09F3F5C
:103B300019F4411101C0982F8F5F8630A9F79F3F7C
:103B400039F0F901E90FF11D97FDFA9562830895A7
:103B500008959C012A5F3F4FFC014281461301C03A
:103B60001282019682179307B9F708950C948F1D5E
:103B70000C94A91D029626E0FC0111922A95E9F702
:103B8000089508950C94C11D83E0809395020C94D0
:103B9000C21D811102C081E001C082E080939502C4
:103BA0000C94C21D0C94C91D81E0809395020C9465
:103BB000C21D0C94D41D08950C94DB1D0C94DC1DC7
:103BC0000C94DB1D0C94DB1D0C94DB1DCF930E9429
:103BD000E21D0E940F130E94E01DC0E08C2F0E9486
:103BE0001A12672B682B692B29F4CF5FC630B1F707
:103BF00080E001C081E0CF91089508951F920F9257
:103C00000FB60F9211248F939F93AF93BF93809120
:103C10009602811113C08091E3039091E403A09177
:103C2000E503B091E6034196A11DB11D8093E30326
:103C30009093E403A093E503B093E603BF91AF91A3
:103C40009F918F910F900FBE0F901F9018958091AC
:103C5000EB03843031F10E94C0031092960220E4FD
:103C600088E190E00FB6F894A895809360000FBEAD
:103C70002093600083B7817F846083BF83B78160B6
:103C800083BF7894889583B78E7F83BF0FB6F894EF
:103C9000A895809160008861809360001092600018
:103CA0000FBE08950E94F0070C94C40382E084BD07
:103CB00093E095BD9AEF97BD80936E0008952FB75E
:103CC000F8948091E3039091E403A091E503B0910F
:103CD000E6032FBF08952FB7F8946091E303709126
:103CE000E4038091E5039091E6032FBF08959C01C2
:103CF0004FB7F8948091E3039091E403A091E5031A
:103D0000B091E6034FBF821B930B089578941F92E6
:103D10000F920FB60F9211248F939F93AF93BF937F
:103D20008091E3039091E403A091E503B091E60351
:103D30000196A11DB11D8093E3039093E403A0932A
:103D4000E503B093E603BF91AF919F918F910F90E0
:103D50000FBE0F901F90189581E08093E00080E2E5
:103D60008093D8001092C9008FE19EE40197F1F78B
:103D700000C0000087E090EBDC018093F403909397
:103D8000F503A093F603B093F7039CE088E10FB628
:103D9000F894A895809360000FBE90936000FFCFC9
:103DA0008091A20208950895CF93DF9321E020939C
:103DB000E9002FEF3091E800215035FD06C035EDC8
:103DC0003A95F1F700002111F5CF2091E80025FF89
:103DD00014C0EC0140E050E068E070E00E94E02098
:103DE0008091E8008E778093E80088E0FE01AAE9E0
:103DF000B2E001900D928A95E1F7DF91CF9108959D
:103E00008093970270939902609398028091EB03DC
:103E1000843001F582E08093E9008FEF9091E80013
:103E2000815095FD06C095ED9A95F1F7000081113E
:103E3000F5CF8091E80085FF0DC040E050E063E0E1
:103E400070E087E992E00E94E0208091E8008E77A0
:103E50008093E8000895BC0184E00C94001FBC012D
:103E600083E00C94001F08958091EA03811109C03A
:103E70000E9471220E94CE228091E2008460809391
:103E8000E20008951092EA0308950C94D91D609100
:103E9000E70381E0611101C080E00C94C41D9091A2
:103EA000EB0381E0943009F080E06091E7030C942B
:103EB000C91D42E061EC81E00E94EA2142E261EC2E
:103EC00082E00E94EA219091EB0381E0943009F0B6
:103ED00080E06091E7030C94D21D8091ED03833064
:103EE00009F461C030F4813071F0823009F49AC075
:103EF00008958A3009F486C08B3009F46CC089308B
:103F000009F0A8C020C08091EC03813A09F0A2C05A
:103F10008091E800877F8093E8008091F003909182
:103F2000F103892B21F468E08AE992E003C060E0A4
:103F300080E090E070E00E942B218091E8008B7778
:103F40008093E80008958091EC03813209F082C0EB
:103F50008091F0039091F103029708F07BC080916B
:103F6000E800877F8093E8008091E80082FD05C02B
:103F70008091EB038111F8CF6DC02091F300809107
:103F8000F20090E0922B029731F48091F1008130A1
:103F900011F0863021F48091F1008093A20280918B
:103FA000E8008B7753C08091EC03813A09F052C04E
:103FB0008091F0039091F103892B09F04BC080911F
:103FC000E800877F8093E8008091E80080FFFCCFC5
:103FD0008091230136C08091EC038132D9F5809124
:103FE000F0039091F103892BA9F58091E800877F78
:103FF0008093E8000E941F228091EE0380932301AA
:104000000C94F0078091EC03813221F58091E80057
:10401000877F8093E8000E941F228091EF038093A6
:10402000A30208958091EC03813AA1F48091E80005
:10403000877F8093E8008091E80080FFFCCF80912B
:10404000A3028093F1008091E8008E778093E800CE
:104050000C941F22089584B7877F84BF0FB6F8940D
:10406000A895809160008861809360001092600044
:104070000FBE90E080E80FB6F894809361009093B3
:1040800061000FBE0C94D41D0E9471220E94CE22AA
:10409000E2EEF0E080818460808378940C94632564
:1040A00087E191E00C942C1D8091EB038530A9F4FD
:1040B0008091EB03853079F40E94271E8091E903FB
:1040C0008823B1F30E94E61D882391F30E94CA2041
:1040D0000E94F007EDCF0C94521E089508950C94A1
:1040E0007120292F332723303105C9F060F42130A6
:1040F000310581F02230310509F044C08BE390E0B6
:104100002FEC34E043C021323105E1F02232310599
:1041100049F138C082E190E02AE035E037C09927C4
:104120008130910549F028F0029761F5E7E8F4E065
:1041300005C0EBECF4E002C0EDEAF4E0849190E01D
:104140009F0124C06115710541F061307105D1F402
:1041500089E090E02AEF34E019C089E090E021EE98
:1041600034E014C06115710541F06130710551F4FE
:1041700082E390E02CE135E009C080E490E02EE499
:1041800035E004C080E090E020E030E0FA013183C7
:104190002083089580E189BD82E189BD09B400FED4
:1041A000FDCF8091D8008F7D8093D8008091E00072
:1041B00082608093E0008091E00081FDFCCF089553
:1041C000CF92DF92EF92FF920F931F93CF93DF93E3
:1041D000EC018B017A010E943E22811133C0E1146F
:1041E000F10439F0F70180819181081B190BC80F88
:1041F000D91FC12CD12C0115110519F18091E800AE
:1042000085FD16C08091E8008E778093E800E11468
:10421000F10449F0F70180819181C80ED91ED18245
:10422000C08285E00FC00E943E22882321F30AC08D
:1042300089918093F10001501109FFEFCF1ADF0A35
:10424000DACF80E0DF91CF911F910F91FF90EF9037
:10425000DF90CF9008952091F2033091F303261759
:10426000370748F06115710539F42091E8002E7781
:104270002093E80001C0B901FC0120E0611571053F
:1042800079F18091EB038823F1F18530F1F1809190
:10429000E80083FD3CC08091E80082FD2EC0809143
:1042A000E80080FFEBCF2091F3008091F20090E0D6
:1042B000922B6115710551F08830910538F42191E8
:1042C0002093F100615071090196F3CF21E0089726
:1042D00009F020E08091E8008E778093E800CECF4F
:1042E0002111CFCF0AC08091EB03882361F0853084
:1042F00061F08091E80083FD0AC08091E80082FFB0
:10430000F2CF80E0089582E0089583E0089581E08F
:1043100008952091F2033091F3032617370748F0F0
:104320006115710539F42091E8002E772093E8009B
:1043300001C0B901FC0120E06115710591F1809186
:10434000EB03882309F440C0853009F43FC0809115
:10435000E80083FD3DC08091E80082FD2FC0809180
:10436000E80080FFE9CF2091F3008091F20090E017
:10437000922B6115710559F08830910540F4249114
:104380002093F1003196615071090196F2CF21E03E
:10439000089709F020E08091E8008E778093E8008C
:1043A000CBCF2111CCCF0AC08091EB03882361F0E1
:1043B000853061F08091E80083FD0AC08091E800BB
:1043C00082FFF2CF80E0089582E0089583E00895AF
:1043D00081E00895982F973068F59093E900981739
:1043E00039F07091EC002091ED005091F00003C085
:1043F000242F762F50E021FD02C09F5FECCF30913B
:10440000EB003E7F3093EB003091ED003D7F309329
:10441000ED003091EB0031603093EB007093EC00D5
:104420002093ED005093F0002091EE0027FDE5CFA2
:1044300080E008958F708093E90081E00895809175
:10444000EC0387FF11C08091E80082FD05C08091D8
:10445000EB038111F8CF11C08091E8008B770BC07E
:104460008091EB03882349F08091E80080FFF8CF2A
:104470008091E8008E778093E80008952091E40011
:104480003091E50095E64091EC00842F817040FF6B
:1044900023C08091E80080FD1DC08091EB0388233C
:1044A00099F0853099F08091EB0085FD11C0409125
:1044B000E4005091E5002417350729F3915011F0DD
:1044C0009A01E1CF84E0089582E0089583E00895A1
:1044D00081E0089580E008954091E80042FFDDCF3B
:1044E00008950E94DF220E94E722E0EEF0E0808142
:1044F00081608083E8EDF0E080818F77808319BC54
:10450000A7EDB0E08C918E7F8C9380818F7E80832D
:104510001092EA0308950F931F93CF93DF930E94A5
:10452000DF220E94E722C8EDD0E088818F77888360
:1045300088818068888388818F7D888319BC1092E8
:10454000EB031092E7031092E9031092E80300EEE8
:1045500010E0F80180818B7F80838881816088836F
:1045600042E060E080E00E94EA21E1EEF0E080813C
:104570008E7F8083E2EEF0E08081816080838081A5
:1045800088608083F80180818E7F8083888180614C
:104590008883DF91CF911F910F910895E8EDF0E0AE
:1045A00080818F7E8083E7EDF0E080818160808371
:1045B00084E082BF81E08093EA030C948B22E8EDD3
:1045C000F0E080818E7F80831092E2000895109247
:1045D000DA001092E10008951F920F920FB60F9229
:1045E00011242F933F934F935F936F937F938F93F8
:1045F0009F93AF93BF93EF93FF938091E10082FF6E
:104600000BC08091E20082FF07C08091E1008B7FA8
:104610008093E1000E9462258091DA0080FF1FC034
:104620008091D80080FF1BC08091DA008E7F80933C
:10463000DA008091D90080FF0DC080E189BD82E160
:1046400089BD09B400FEFDCF81E08093EB030E9499
:10465000341F05C019BC1092EB030E94421F8091C9
:10466000E10080FF19C08091E20080FF15C08091B9
:10467000E2008E7F8093E2008091E200806180936F
:10468000E2008091D80080628093D80019BC85E058
:104690008093EB030E94471F8091E10084FF30C0AC
:1046A0008091E20084FF2CC080E189BD82E189BD58
:1046B00009B400FEFDCF8091D8008F7D8093D80093
:1046C0008091E1008F7E8093E1008091E2008F7EF7
:1046D0008093E2008091E20081608093E20080910B
:1046E000E703882311F084E007C08091E30087FD91
:1046F00002C081E001C083E08093EB030E944F1F62
:104700008091E10083FF29C08091E20083FF25C0F2
:104710008091E100877F8093E10082E08093EB034A
:104720001092E7038091E1008E7F8093E1008091F9
:10473000E2008E7F8093E2008091E20080618093AE
:10474000E20042E060E080E00E94EA218091F00017
:1047500088608093F0000E94451FFF91EF91BF9108
:10476000AF919F918F917F916F915F914F913F9109
:104770002F910F900FBE0F901F9018951F920F92C0
:104780000FB60F9211242F933F934F935F936F9324
:104790007F938F939F93AF93BF93CF93DF93EF93C9
:1047A000FF93C091E900CF708091EC00D82FD170B9
:1047B00080FDD0E81092E9008091F000877F80931F
:1047C000F00078940E9402241092E9008091F00099
:1047D00088608093F000CD2BCF70C093E900FF91EB
:1047E000EF91DF91CF91BF91AF919F918F917F9189
:1047F0006F915F914F913F912F910F900FBE0F904E
:104800001F9018951F93CF93DF93CDB7DEB7AA976C
:104810000FB6F894DEBF0FBECDBFECEEF3E0809193
:10482000F100819323E0E43FF207C9F70E946D1F76
:104830008091E80083FF2EC18091EC039091ED03FD
:10484000492F50E04A30510508F024C1FA01EE59D1
:10485000FF4F0C94D625803821F0823809F01AC118
:1048600008C08091E8039091E903992389F0826060
:104870000FC08091F0038F70873008F00BC18093D8
:10488000E9008091EB0085FB882780F91092E90010
:104890009091E800977F9093E8008093F100109248
:1048A000F100D1C0282F2D7F09F0F4C0882319F022
:1048B000823061F0EFC08091EE03813009F0EAC0F0
:1048C000933009F080E08093E9032EC08091EE03DD
:1048D00081112AC08091F0038F702FEF280F2630AE
:1048E00008F0D8C08093E9002091EB0020FF1CC0A5
:1048F000933021F48091EB00806214C09091EB0022
:1049000090619093EB0021E030E0A90102C0440FD8
:10491000551F8A95E2F74093EA001092EA008091D1
:10492000EB0088608093EB001092E9008091E80032
:10493000877F8093E8000E941F22ACC08111AAC02B
:104940001091EE031F778091E3008078812B809394
:10495000E3008091E800877F8093E8000E941F2297
:104960008091E80080FFFCCF8091E3008068809315
:10497000E300111102C082E001C083E08093EB03E9
:1049800089C08058823008F085C08091EE039091F4
:10499000EF038C3D53E0950779F583E08A838AE243
:1049A00089834FB7F894DE01139620E03EE051E290
:1049B000E32FF0E050935700E49120FF03C0E2950D
:1049C000EF703F5FEF708E2F90E0EA3010F0C796E7
:1049D00001C0C0968D939D932F5F243149F74FBF3F
:1049E0008091E800877F8093E8006AE270E0CE0162
:1049F00001960E942B2116C06091F0037091F10383
:104A0000AE014F5F5F4F0E946F20BC01892B09F4FC
:104A100041C09091E800977F9093E80089819A8146
:104A20000E9489218091E8008B778093E80032C052
:104A3000803881F58091E800877F8093E80080913D
:104A4000E7038093F1008091E8008E7772CF8111A7
:104A500021C08091EE039091EF0399270297D4F43F
:104A60008091E800877F8093E8008091EE03809337
:104A7000E7030E941F228091E703811106C0809105
:104A8000E30087FD02C081E001C084E08093EB0376
:104A90000E94591F8091E80083FF0AC08091E800BE
:104AA000877F8093E8008091EB0080628093EB0029
:104AB000AA960FB6F894DEBF0FBECDBFDF91CF919F
:104AC0001F9108950895CF938091EB038823A1F05F
:104AD000C091E900CF709091EC00892F817090FD1A
:104AE00080E8C82B1092E9008091E80083FD0E94C5
:104AF0000224CF70C093E900CF91089587FB082E60
:104B0000062687FD819567FD61950E940D260EF4AE
:104B1000919507FC81950895AA1BBB1B51E107C025
:104B2000AA1FBB1FA617B70710F0A61BB70B881F3D
:104B3000991F5A95A9F780959095BC01CD010895CC
:104B400097FB072E16F4009407D077FD09D00E943A
:104B50008C2507FC05D03EF4909581959F4F0895D4
:104B6000709561957F4F0895A1E21A2EAA1BBB1B79
:104B7000FD010DC0AA1FBB1FEE1FFF1FA217B30729
:104B8000E407F50720F0A21BB30BE40BF50B661F3F
:104B9000771F881F991F1A9469F760957095809503
:104BA00090959B01AC01BD01CF010895EE0FFF1F51
:104BB0000590F491E02D09940E94E425332312F42A
:104BC0008A1B9B0B0C94F525A29FB001B39FC001DB
:104BD000A39F700D811D1124911DB29F700D811D29
:104BE0001124911D08950E94E425B7FF0895821BAA
:104BF000930B08950E94E425A59F900DB49F900DFE
:104C0000A49F800D911D11240895B7FF0C94FA25DF
:104C10000E94FA25821B930B0895991B79E004C02A
:104C2000991F961708F0961B881F7A95C9F78095EB
:104C30000895FC014150504030F001900616D1F724
:104C40003197CF010895882799270895FB01DC014A
:104C500004C08D910190801921F441505040C8F753
:104C6000881B990B0895F999FECF92BD81BDF89AE2
:104C7000992780B50895A6E1B0E044E050E00C9497
:104C80006D26A8E1B0E042E050E00C946D26262F9E
:104C9000F999FECF92BD81BDF89A019700B4021632
:104CA00039F01FBA20BD0FB6F894FA9AF99A0FBEE0
:104CB00008950396272F0E9448260E944726252FF5
:104CC0000E944826242F0C9448260196272F0E94E4
:104CD00048260C944726DC01CB01FC01F999FECF54
:104CE00006C0F2BDE1BDF89A319600B40D92415074
:0A4CF0005040B8F70895F894FFCF84
:104CFA00C8005102010102005800585801191A1B34
:104D0A001C1D1E1F202122D01ED41E331F2F1F2B15
:104D1A001FD31E01E200E900EA00B500B600B700A1
:104D2A00CD008301CC008A01920194012102230261
:104D3A0024022502260227022A02B300B4006F00C9
:104D4A007000818283E200E900EA00B500B600B78C
:104D5A0000CD008301CC008A019201940121022333
:104D6A000224022502260227022A02B300B4006F97
:104D7A0000700081828330313233F4F5F6F736352C
:104D8A00973496F0916694939237F16795000102F1
:104D9A000202020606060909090909090F0F0F0F7F
:104DAA000F0F15151518191919191919191919198A
:024DBA002324B0
:00000001FF
